:020000040000FA
:1000000085018601831634287E2882070D341A3430
:1000100033344934663483349934B434D134820768
:100020000F341D343834513471349134AA34C73408
:10003000E7348207083410342034403480340034EC
:1000400000340034003401348207003400340034BA
:1000500000340034403480340134023400348207E8
:100060000034043408341034003085000630860033
:100070001030980020308C00831207309F004030F1
:100080008B00C0309800F1010930F600F001F20158
:10009000F70106148B17181670186F280930F10035
:1000A000F103F11B5F28710805207202031C502820
:1000B00071080F20720203196128031C612809309E
:1000C000F1007108F606F60003197B283C3085051F
:1000D0007108192086007108242085047B28720885
:1000E0000339F706F70003197B28E3308505770805
:1000F0002F2085047B28630000004C28F500030EA8
:10010000F4007010181870141A08F200740E8300AE
:06011000F50E750E09005A
:02400E00503F21
:00000001FF
